:020000040800F2
:10500000E01F0020D550000855900008B386000826
:105010000000000000000000000000000000000090
:10502000000000000000000000000000159C0008C7
:105030000000000000000000FD990008559D0008D8
:10504000E7500008E7500008E7500008E750000864
:10505000E7500008B55C0008E7500008E75000087A
:1050600000000000E7500008C15B0008E75000089E
:10507000E7500008858B000800000000E75000089A
:1050800000000000E75000080000000000000000E1
:10509000E750000800000000E7500008E750000853
:1050A000E7500008E7500008E7500008E9A70008AB
:1050B000E7500008E7500008000000000000000072
:1050C0000348854600F0C6FC00480047C9B8000800
:1050D000E01F00200448804704480047FEE7FEE741
:1050E000FEE7FEE7FEE7FEE7159E0008C150000858
:1050F00030B50B46014600202022012409E00D4670
:10510000D5409D4205D31D469540491B25469540F7
:1051100040191546521E002DF1DC30BD70B500243B
:105120002546002801DA01244042002901DA012540
:105130004942FFF7DDFFAC4200D04042002C00D0D6
:10514000494270BDF0B51FB40646002082B0054646
:105150004024019100901BE0019922460F46304601
:1051600000F062FB049A059B801A994110D3104607
:105170001946224600F048FB361A8F410197224615
:1051800001200021009F00F03FFB38184D410090A6
:105190002046641E0028DFDC019B00982946324629
:1051A00007B0F0BD03460B439B0703D009E008C9D5
:1051B000121F08C0042AFAD203E00B780370401CC7
:1051C000491C521EF9D27047D2B201E00270401C55
:1051D000491EFBD270470022F6E710B513460A4677
:1051E00004461946FFF7F0FF204610BD30B50446CF
:1051F0000020034600E05B1C934203D2E05CCD5CE0
:10520000401BF8D030BDF8B502464A40D40F4200EA
:105210004B0052085B089A4202D2024608461146E9
:105220004A0023D0C30D4A00DDB2120EAD1A202D64
:1052300035DA49020126490AF6058A19002C00D000
:10524000524220214F1B1146B9402A411018C20D6D
:105250009A4221D0002C17D0012D08DCDA05801AE3
:10526000D20F8019D207DBB200F00AFBF8BDDA05D5
:10527000801A012340001B06C01880185A4280186B
:10528000CA0F1043490007E04908C2071143DA0575
:10529000801A80194008801800F0EAFAF8BD610011
:1052A0000122511A001BF7E70122D2075140AAE759
:1052B0000122D2075040A6E770B502464A40D50FFA
:1052C00040004A00ED0740085208002814D0002A88
:1052D00012D0C40DD30D41020120C0055202490A6B
:1052E000520AE41A091812187D34914201D3641C41
:1052F00000E04900002C01DA002070BD002391423B
:1053000001D3891A0343400849000028F7D1002936
:105310000AD0914202D10121C90705E0914201D290
:10532000012101E00121C943E005C018401900F046
:105330009FFA70BDF0B507460846584087B0C00FC9
:10534000049048000E46590040084908BC1A88419C
:1053500005D2384631461E4617460B4602465800CF
:10536000400810434CD0300D039040055900400DCB
:10537000490D0590401A0290402872DA1803012165
:10538000000B09050843019004980092002805D0FD
:1053900001995242002088410092019002984021D8
:1053A0000A1A0199009800F02FFA05460C466B4640
:1053B00007CB00F04AFAC0197141039A0E0D002381
:1053C000D71756401A467A40164344D0049A002A0A
:1053D0002DD0029A012A039A15DC1205C01A9141B8
:1053E00001263605001C7141D20F059ED20700939D
:1053F000019202962A46234600F088FA07B0F0BDD3
:1054000038463146FAE71605224A0F46B218C01A46
:10541000B74101210905001C4F4100187F41114689
:1054200018187941E20F10436D19644113E0E20747
:105430006D0815436408C2071443039A0126120538
:10544000C01A91413605001C7141CE074008304317
:105450004908C01851412A46234600F04AFACDE7D0
:10546000FFE7049801224000C117121A00238B4164
:1054700004983146C417381AA141EEE730B401242C
:10548000E407634030BC55E730B40124E4076140D1
:1054900030BC4FE70000E0FFF0B51FB488B00B99B7
:1054A0000998002448400999C00F4900490809910A
:1054B000C0070B990090490049080B910999089879
:1054C000A64608431CD00B990A98084318D009989F
:1054D00001244000420D4800410D099824050003B5
:1054E000000B204309900B980003000B20430B9006
:1054F00050181C494018002201901446104605E03F
:10550000002001460DB0F0BD032801DA034600E09B
:1055100003239C46C11A0AAE0AE05F0008ADED5BAA
:105520004F00F75B7D430027AA187C41491C5B1E96
:105530006145F2DD410004AB5A522104120C0A43CA
:10554000240C401C0828DFDB01980290009970466B
:1055500001910090059B049A0799069800F0D6F9EE
:10556000D0E700000DFCFFFFF0B50C465C4085B0B5
:10557000E40FE40703944C000026640859009446A5
:10558000490802460296224321D062460A431ED0B1
:105590006200570D4A000E032303550D01240246F5
:1055A0002C492405781B1B0B360B4018234326433C
:1055B000614600901C46501AB44103D30098401C29
:1055C000009002E0921800985B41002803DA002066
:1055D000014605B0F0BD00200121090507468646B9
:1055E00011E064461D46141BB54106D36546521BA7
:1055F000B341744607430C43A646CD07400849080B
:10560000284392185B4105460D43EAD110461843E2
:1056100013D06046194650407140084306D060469A
:10562000101AB34106D20122002306E00022012312
:10563000DB0702E00122D2435310009874460105B3
:10564000381C6141029C039D0019694100F051F929
:10565000BFE70000FD03000010B5002296231146AD
:1056600000F00EF910BD00000EB5C217C10F50407A
:10567000CA0740180021054B0293019200910A4687
:105680000B4600F043F903B000BD000033040000F6
:105690000EB505490291002100910A460B46019181
:1056A00000F034F903B000BD3304000041004002B3
:1056B0000122400AD205090E80187F2901DA002054
:1056C0007047962903DC9622511AC84070479639D4
:1056D0008840704770B5CD0F4A0009030123090BBC
:1056E0001B0519430B4BED070024520D9A4201DABA
:1056F000002070BD074B34339A4203DC9A1A00F045
:1057000093F802E00449511888402C43F1D04042FC
:1057100070BD0000FF030000CDFBFFFF4A0009033E
:105720000123090B1B051943094B10B5520D9A4271
:1057300001DA002010BD064B34339A4203DC9A1A7A
:1057400000F072F810BD03495118884010BD0000E8
:10575000FF030000CDFBFFFFC20FD207400040084F
:105760000BD0C10D0723DB01C91840020905400A0F
:105770001143C2084007114370470020014670479B
:1057800010B5002904DB0124E40740428C41214686
:10579000002B04DB1C460123DB075242A341994244
:1057A00000D1904210BD0000CB0FDB07490010B5BF
:1057B000490802460A4307D00A0D07240903E401F9
:1057C000090B121B002A01DC002010BDC900440F88
:1057D0000C43C100E018D205801800F049F810BD54
:1057E0000122D207002800DB101A002900DB511A21
:1057F000814270470122D207002800DB101A0029DD
:1058000000DB511A8842704710B5202A04DB01469C
:10581000203A9140002010BD914020239C1A03465D
:10582000E3401943904010BD10B5202A04DB084620
:10583000203AD040002110BD0B46D340D040202458
:10584000A21A91400843194610BD10B5202A06DB64
:10585000CB170846203A1041C1170B4306E00B4610
:105860001341D0402024A21A91400843194610BD8C
:10587000002904DA401C490001D14008400070476B
:1058800070B40024050C05D11024000402D10029B5
:1058900021D01124050E01D100020834050F01D1D9
:1058A0000001241D850F01D18000A41C002801DB0C
:1058B0004000641C002908D020252E1B0D46F54011
:1058C000A14000D001212943084301061B1B000A07
:1058D000DB1D02D5002070BC7047DB05181880184E
:1058E0000029F8DA401C4900F5D170BC400840009E
:1058F000704710B5002B08DA0024401C6141921853
:105900005B411A4301D14008400010BDF0B51FB4FF
:1059100082B005460C0003D0084605F075F802E099
:1059200005F072F820300246009021462846FFF725
:105930006BFF049B059A04460F4618431143084326
:1059400014D0184610431BD0009840210A1A18465C
:105950000599FFF769FF05460E46009A05990498D8
:10596000FFF752FF084305D0012004E020463946E6
:1059700007B0F0BD0020C11705430E432C43374349
:1059800000990E986305401A7905E40A00220C4339
:10599000FD0A0A3002D500200146E9E70105101989
:1059A00069410C9C0D9D00196941FFF7A2FFDFE7DB
:1059B000F8B50546480040080C46284304D060006E
:1059C000184A400D904201DD2846F8BD1549353989
:1059D000884210DC88420BDB290D20030843290391
:1059E000014305D0E00F1049C00741180020F8BD61
:1059F00000200146F8BD161A4020821B2846214689
:105A0000FFF702FF07460091284621463246FFF77E
:105A10000BFF3A46009BFFF76CFF3246FFF7F4FEA0
:105A2000F8BD0000330400000000F03F10B500296D
:105A300004DB0124E40740428C412146002B04DBB7
:105A40001C460123DB075242A3418B4200D1824214
:105A500010BD0000064C0125064E05E0E36807CCAA
:105A60002B430C3C98471034B442F7D3FFF72CFB80
:105A700000BD000820BD000870B58C180578401CDA
:105A80006B075B0F01D10378401C2A1106D1027805
:105A9000401C03E006780E70401C491C5B1EF9D1C7
:105AA0002B0705D40023521E0DD40B70491CFAE7B6
:105AB0000378401CCB1A921C03E01D780D70491C22
:105AC0005B1C521EF9D5A142D8D3002070BD000046
:105AD00038B50446074908480068FFF709FB6043EA
:105AE000009002E00098401E009000980028F9D134
:105AF00038BD000040420F007801002070B5044618
:105B00000025206880688007800F012807D1206861
:105B10000068C007C00F002801D0012000E000206D
:105B2000002839D1206880681C490840002801D12C
:105B3000012000E00020002809D1606D10210843F9
:105B40006065A06D01210843A065012070BD20683B
:105B5000806801210843216888600120FFF7B8FFB1
:105B600001F040FA05460EE001F03CFA401B0A281D
:105B700009D9606D102108436065A06D01210843BB
:105B8000A0650120E2E720680068C007C00F01217E
:105B9000484048400028E7D00020D7E717000080A1
:105BA00010B502460B460020002103E0545C241887
:105BB000A0B2491C9942F9D3C443A0B210BD000061
:105BC00010B5034800F00CFF024800F009FF10BDBB
:105BD0007C1B0020341B002030B51C25446C2C405D
:105BE0000125A540046C6560046863608468102C1E
:105BF00004D10468A2600468E16003E00468A16065
:105C00000468E26030BD000001201749487202209C
:105C100016494872032016494872042015494872F3
:105C2000114815490A784271497881711048124922
:105C30000A784271497881710C480F490A7842709C
:105C4000497881700B480C490A7842704978817014
:105C50000A4809490A7842704978817006490A78E9
:105C60004271497881717047AC1500200A160020F6
:105C7000CE150020C01500203C0100202016002079
:105C800010B503F09BFF202004F052F8012005F02E
:105C9000D7FA002004F04CF8044805F03FF9044816
:105CA00005F07EFC002005F0BBFC10BD610000206B
:105CB0008380000010B501210520000701F082F962
:105CC000002802D000200A4908600221094801F09A
:105CD00079F9002805D1084800880A214843074976
:105CE0000880012001F068F8022001F065F810BD7D
:105CF00070010020000400505801002068010020BD
:105D00007047000000210A4A51610A49496801228E
:105D100052021143074A5160114649680822114353
:105D2000044A51600021C209D2011160704700008D
:105D3000C41B0020002002407FB504460D46002011
:105D4000039000F0F1FF002000900194E809029018
:105D500003A9684600F06AFF002804D000F0ACFFF9
:105D6000002004B070BD00F0A7FF0120F9E710B5D6
:105D70000346002002E01C5C0C54401C9042FAD305
:105D800010BD0000002039498969FF22013211400D
:105D9000914208D13649496902221143344A51617E
:105DA000FF21013108433149896901225202114022
:105DB000914208D12E494969012211432C4A51616F
:105DC00001214902084329498969012292021140AF
:105DD000914208D12649496908221143244A516158
:105DE000012189020843214989690122D202114017
:105DF000914208D11E494969042211431C4A51614C
:105E00000121C9020843194989690122520311403D
:105E1000914208D11649496910221143144A51612F
:105E200001214903084311498969012252041140A3
:105E3000914207D10E494969202211430C4A516110
:105E40002021084309498969012212041140914225
:105E500008D10749496940221143054A516101218E
:105E6000090408430149886170470000002002408E
:105E7000C41B002070B5044601F0B4F805460BE0E1
:105E8000601C002808D0002C04D001F0ABF8401BA7
:105E9000A04201D9032070BD1F488069C007C00F10
:105EA0000028EDD11C48806902210840022801D158
:105EB0001949886118488069FF21013108408842EA
:105EC00023D0154880694900084088421DD01248F7
:105ED000806949000840884217D00F48806949000E
:105EE0000840884211D00C488069890008408842E7
:105EF0000BD00948806909010840884205D006484E
:105F0000806949100840884203D1FFF73BFF012018
:105F1000C1E70020BFE7000000200240F0B585B0D7
:105F200006460F4614460025029601970020009071
:105F300000F0FAFE13E00198006803900220039A33
:105F4000029900F0C9FE00900098002800D008E0F7
:105F50000298001D02900198001D01902D1DA54280
:105F6000E9D300BF00F0A8FEA54202D2002005B090
:105F7000F0BD0120FBE700000246002108E04800D8
:105F8000064B185A904201D108467047481CC1B2CE
:105F9000034800788142F2DB00BFF6E71A180020C0
:105FA00028010020FEB50C4801F0D4F980B202901F
:105FB0000298FFF76DFB0446084A094BFFF76CFA9D
:105FC0000022084B01910090FFF7CEFA0646FFF73A
:105FD000A5FB80B2FEBD00002C1A0020F853E3A5FB
:105FE0009B843E4000408F4070B586B05748007893
:105FF000002803D000205549087002E001205349D1
:106000000870534851490A78427049788170514963
:106010000A7842714978817105204D49487296206D
:1060200005F0ACFA4B20C00005F0C4FA0022484944
:106030000C2005F0C1FB00210C2005F0D1FB022053
:1060400005F0F6FA00BF00210F2005F0EFF94249F4
:106050000860424908400028F5D03F480068401CCD
:10606000002801D103F034F83B480068012189037E
:106070000840002858D08122D20100210F2005F0CD
:1060800054FB0021102005F0D1F94606760E31466A
:106090000022334805F01AFA3148407A052853D1D6
:1060A00002222C492E48401DFFF7A0F800284BD1B2
:1060B0002B48807A2B49087004222949491C2A4818
:1060C000FFF770F82848006800F062F82749088058
:1060D00024480078420022490B312548FFF762F836
:1060E00020480078801CFFF7BFFA0446214A224B63
:1060F000FFF7D2F90191009004F05AFE00221F4BE5
:1061000003910290FFF716F905910490FFF706FB43
:106110001B490880154800880988484319490880A8
:106120000220194908700FE0104908880988491EA3
:106130000E4B198015490988FEF7F0FF10480088BA
:10614000414388B20F49088006B070BD330100207A
:10615000201600203C0100207000002000D02724E1
:1061600070160020280100202C010020FC000020D7
:106170001A180020333333333333D33F0000F03F5A
:106180004E0100204A010020600000205001002044
:1061900070B5064600F030F805462846E917C90EE6
:1061A000091849114901691ACCB209E03046E040AA
:1061B000C007C00F002801D1204670BD601CC4B2CA
:1061C0000C4800888442F1DB012409E03046E040BD
:1061D000C007C00F002801D12046EEE7601CC4B202
:1061E000044800888442F1DB02480078401EC0B2B7
:1061F000E3E700005001002070B50025002409E00D
:1062000000F00CF8C6B2F007C00FA0402843C5B29A
:10621000601CC4B2082CF3DB284670BD10B50B48D7
:1062200000F074FB0A21094800F0FAFA074800F070
:10623000A1F9012149020840884204D1034800F035
:106240009CF980B210BD00BFFCE70000D01900200F
:10625000F0B587B000220121424800F0BCFEFFF7F4
:10626000DDFF0546FFF7F8F904463F49FFF724F83C
:106270003E490860012211463A4800F0ACFE3B4816
:106280000068FFF769FA04460022394BFFF778FAF5
:106290005ED838480078002821D0002035490870A1
:1062A000FFF7BCFF0546FFF7D7F904462E49FFF775
:1062B00003F82E49086008460068FFF74DFA0446C7
:1062C00000222B4BFFF7DAF800222B4B05910490AC
:1062D000FFF7E2F80646FFF767FA28490860234807
:1062E0000068FFF739FA06460022214BFFF7C6F88F
:1062F0000446234A234BFFF7CFF8039102901F482F
:106300000068FFF729FA04461D4A52421E4BFFF768
:10631000C3F801910090039B029AFFF70BF80591D7
:106320000490FFF741FA15490860184913480068BE
:10633000FFF760FA02D215481049086000210F48A3
:106340000068FFF74DFA06D200200C49086002E011
:1063500000200A49086009480068FFF7A7F9C0B2A1
:1063600007B0F0BD0004005000401B44280000208E
:1063700000000C403000002000E064402C000020B1
:106380003333333333B33040CCCCEC3F0000C8421E
:10639000F8B5044600250026002700BF5020005D08
:1063A000012801D10220F8BD01215020015500BF74
:1063B000206880688007800F012806D12068006867
:1063C0000840002801D0012000E00020002841D131
:1063D000606DFF2101318843022108436065206818
:1063E000C0688707BF0F2068C068800880002168E8
:1063F000C860206880680121C90708432168886057
:1064000000F0F0FD064611E000F0ECFD801B0A28CC
:106410000CD9606D0221884310210843606500BFDC
:1064200000215020015500BF0120BCE72068806892
:10643000C00FC0070121C9078842E5D02068C068A5
:1064400038432168C860606D0221884301210843F8
:10645000606504E0606D202108436065012500BF90
:1064600000215020015500BF28469CE770B5044626
:106470000D4600BF5020005D012801D1022070BDF3
:1064800001215020015500BF206880680421084088
:10649000800800280AD0606D20210843606500BF95
:1064A00000215020015500BF0120E8E72D49686810
:1064B000884229D02068806A29684903490B08432B
:1064C0002168886228684003400B27490840012161
:1064D0008904884208D12548806849010843234936
:1064E00088600A20FFF7F4FA28684003400B20492F
:1064F00008400121490488422CD11C488068490188
:1065000008431A49886025E02068806A29684903A1
:10651000490B88432168886228684003400B124970
:10652000084001218904884205D11048806849014A
:1065300088430E49886028684003400B0C49084096
:1065400001214904884205D10848806849018843EF
:106550000649886000BF00215020015500BF00207F
:106560008DE70000011000000000044800270140F2
:10657000000002440146486D704701460868006CFF
:106580007047000010B50446002C01D1012010BD59
:10659000606D002806D1A0650021502001552046DD
:1065A00000F00EF9606D10210840102806D0206818
:1065B000806804210840800800280AD0606D1021FE
:1065C0000843606500BF00215020015500BF012035
:1065D000DDE7606DFF2101318843022108436065DA
:1065E000206880688007800F012807D12068006834
:1065F000C007C00F002801D0012000E000200028C3
:106600003AD100BF032189076068884207D0494218
:106610006068884203D04900606888420CD12068D5
:10662000006980008008216808612068006961684D
:1066300008432168086112E0206800698000800832
:10664000216808615C4880680F21890488435A49A1
:10665000886008468068616808435749886000BFC1
:106660002068C068182188432168C8602068C06815
:10667000A16808432168C8604F4880680121490625
:1066800088434D49886008468068A18E49060843C2
:10669000494988602068806801210907084000286E
:1066A00004D1206880680843216888602068C06839
:1066B000424908402168C8602169E068022901D187
:1066C000042100E0002108432021095D490308431B
:1066D0002C21095D49000843216B0843A169890306
:1066E0000843E169C90308432168C9680843216870
:1066F000C860FF21C231606A884207D0A16A606A1F
:1067000008432168C96808432168C8602120005DEA
:10671000012813D12020005D002807D12068C0681F
:106720000121090408432168C86007E0606D202149
:1067300008436065A06D01210843A065E06B012856
:1067400017D120680069FF2189008843216808610A
:10675000216C606C0843A16C0843216809690843F7
:1067600021680861206800690121084321680861E7
:106770000BE020680069C007C00F002805D0206822
:106780000069400840002168086120684069C0082D
:10679000C0002168486120684069A16B08432168F6
:1067A00048610020A065606D0221884301210843F3
:1067B00060650020EBE60000002701401902FEFFA3
:1067C00010B586B00446142101A8FEF704FD124955
:1067D000206888421ED11148406B491508430F4973
:1067E000486300BF0846C06A012108430B49C862DC
:1067F0000846C06AC007C00F009000BF00BF02205B
:106800000190032002900020039001A905200007B9
:1068100000F0E2FA06B010BD002401400010024072
:10682000F8B504460D46002600276069082801D106
:10683000082711E02068C068C007C00F00280AD0F0
:10684000606D20210843606500BF00215020015584
:1068500000BF0120F8BD0C2700F0C4FB064614E081
:10686000681C002811D0002D04D000F0BBFB801B59
:10687000A8420AD9606D04210843606500BF002169
:106880005020015500BF0320E4E72068006838402D
:106890000028E5D0606D0121490208436065206849
:1068A000C068032189020840002826D12020005D0D
:1068B000002822D1206800680821084008281CD13F
:1068C0002068806804210840800800280DD12068D5
:1068D00040680C21884321684860606DFF210131C8
:1068E000884301210843606507E0606D202108436B
:1068F0006065A06D01210843A065A069002802D150
:106900000C20216808600020A4E7000070B5044650
:1069100000252068806804210840800800282BD1C9
:1069200000BF5020005D012801D1022070BD01216F
:106930005020015500BFE069012803D02046FFF731
:10694000DDF80546002D18D1606D0D490840FF2186
:106950000131084360650020A06500BF0021502080
:10696000015500BF1C202168086020688068042150
:1069700008432168886000E002252846D6E7000029
:10698000FEF1FFFF70B5044600252520005D0228BA
:1069900003D00420E063012520E0206800680E2178
:1069A000884321680860206800684008400021682A
:1069B00008601C21606C084001218140206C41600E
:1069C00001212520015500BF00212420015500BFD1
:1069D000A06B002802D02046A16B8847284670BDD6
:1069E00070B50446206C0568206806681C20616C40
:1069F000014004208840284000281DD00420304059
:106A0000002819D02068006820210840002805D1FE
:106A10002068006804218843216808601C21606C9C
:106A2000084004218140206C4160206B00285AD02E
:106A30002046216B884756E01C20616C01400220F3
:106A400088402840002825D002203040002821D04E
:106A50002068006820210840002808D120680068CC
:106A60000A218843216808600121252001551C2145
:106A7000606C084002218140206C416000BF002111
:106A80002420015500BFE06A00282CD02046E16A8E
:106A9000884728E01C20616C01400820884028407D
:106AA000002820D00820304000281CD02068006832
:106AB0000E218843216808601C21606C0840012178
:106AC0008140206C41600120E063012125200155B7
:106AD00000BF00212420015500BF606B002802D0B8
:106AE0002046616B884770BD70B50446002C01D10B
:106AF000012070BD244A2168881A1421FEF7F8FA93
:106B00008000606420480838206402212520015557
:106B1000206805681D480540E168A06808432169B0
:106B2000084361690843A1690843E1690843216A90
:106B3000084305432068056001218903A068884255
:106B400017D011487830806A1C22616C11400F22E6
:106B50008A4090430C49783188621C22616C114054
:106B60006068884008497831896A08430649783165
:106B700088620020E06301212520015500212420A6
:106B800001550020B5E70000080002400F80FFFF1C
:106B9000F8B504460D4616461F460020009000BF7B
:106BA0002420005D012801D10220F8BD012124200C
:106BB000015500BF2520005D01282DD1022125208F
:106BC00001550020E063206800684008400021680B
:106BD00008603B46324629462046FEF7FDFF206B03
:106BE000002806D0206800680E210843216808604C
:106BF0000BE0206800680421884321680860206851
:106C000000680A21084321680860206800680121A3
:106C100008432168086006E000BF002124200155D8
:106C200000BF022000900098BFE70000F8B50446BE
:106C30000E460127002500BF1C48007C012801D119
:106C40000220F8BD01201949087400BF1848FFF759
:106C500011F90746002F22D1401E3060656817E009
:106C60002846FFF74FF81248FFF704F90746114886
:106C70004068082188430F49486008464068491524
:106C800088430C494860002F01D0356006E080350C
:106C9000A068C00161684018A842E1D800BF00BFE9
:106CA00000200249087400BF3846CAE7C41B002010
:106CB00050C30000002002400648406802210843FB
:106CC000044948600846406801210843014948607A
:106CD0000020704700200240F8B507460C461546D4
:106CE000012600BF0E48007C012801D10220F8BD1A
:106CF00001200B49087400BF0A48FFF7BBF806469D
:106D0000002E06D10649486125600648FFF7B2F813
:106D1000064600BF00200249087400BF3046E6E77F
:106D2000C41B002050C300001D484068C007C00FAE
:106D3000002816D000BFEFF31080014600BF72B6E6
:106D40001848174AD0601848D06000BF81F31088F7
:106D500000BF10464068C007C00F002801D00120C6
:106D600070470F48406802221040022815D100BF2A
:106D7000EFF31080014672B60C48094A10610C48C6
:106D80001061084680F3108800BF10464068022258
:106D90001040022801D10120E2E70020E0E70000D6
:106DA00000200240EFCDAB8905040302BFAE9D8CED
:106DB000161514137047000010B5044605484069C5
:106DC0002040002804D0034844612046FFF7F2FF2A
:106DD00010BD00000004014070B5034600220024ED
:106DE0000020DAE0012696400D6835402C46002C44
:106DF00077D04D68022D02D04D68122D15D1D508DF
:106E0000AE001D462035A8595507EE0E0F25B5409A
:106E10000646AE4330465607F60E0D69B540284388
:106E2000D508AD001E46203670514D68012D08D0A2
:106E30004D68022D05D04D68112D02D04D68122DE0
:106E400018D1986856000325B5400646AE43304633
:106E50005600CD68B5402843986058680125954094
:106E60000646AE43304610264D6835402D09954004
:106E700028435860186856000325B5400646AE43BF
:106E800030460D79AD07AD0F5600B5402843186068
:106E9000D86856000325B5400646AE433046560036
:106EA0008D68B5402843D860012636074D683540C7
:106EB000B54271D13C4D6D6B012635433A4E756339
:106EC0003A4D9608B600A85995072E0F0F25B540E4
:106ED0000646AE43304605252D07AB4202D10025BC
:106EE00015E059E0324DAB4201D101250FE0314DA3
:106EF000AB4201D102250AE02F4DAB4201D103255F
:106F000005E02E4DAB4201D1052500E00625960790
:106F1000360FB5402843254D9608B600A851284D98
:106F200028680546A5432846012636044D683540A5
:106F3000B54202D1054625432846214D28606868A0
:106F40000546A5432846012676044D683540B542DE
:106F500002D1054625432846194D6860A8680546B4
:106F6000A5432846012636054D683540B54202D175
:106F7000054625432846124DA860E8680546A54306
:106F80002846012676054D683540B54202D10546B2
:106F9000254328460A4DE860521C0D68D540002D57
:106FA00000D01FE770BD0000001002400800014043
:106FB0000004005000080050000C0050001C00505D
:106FC00000040140024613690B40002B01D0012050
:106FD00000E000207047002A01D0816100E081625A
:106FE00070470000014800687047000074010020ED
:106FF00002480068401C0149086070477401002085
:1070000010B500240848006840210843064908607C
:10701000002000F00BF8002801D0012401E000F06E
:10702000CFF9204610BD00000020024070B5044694
:1070300000257D21C90009480068FEF759F8064679
:1070400001F07EF8002801D0012504E0002221464D
:10705000501E00F0DDF9284670BD000078010020C8
:107060007047704770B5054619480078401C1849AC
:10707000087001201749087017480088401C1649FD
:1070800008801648008802F009FE1549C888FEF7F6
:10709000E3FA06461349FEF70FF904461248016861
:1070A0002046FEF7B0F8104908600D49488FFEF7FA
:1070B000D3FA04460C4801682046FEF791FB05D23E
:1070C0000A480078002801D004F07AFC70BD000066
:1070D0006C01002049010020620100204A010020CB
:1070E000AC0D002000007A44700100205E010020F9
:1070F000704710B50446002C01D1012010BD0221BB
:107100002E200155204601F045FD204600F0F4F800
:1071100000212E20015500BF2D20015500BF002069
:10712000ECE77047704710B5044620680068C00758
:10713000C00F01214840484000280CD020688068DA
:10714000084048404840002805D001202168486098
:107150002046FFF787FF20680068022108404008AA
:1071600000280BD02068806808404008002805D01F
:107170000220216848602046FFF772FF20680068FF
:1071800004210840800800280BD02068806808404F
:107190008008002805D0042021684860204600F0BF
:1071A0000DF92068006808210840C00800280BD0AD
:1071B000206880680840C008002805D008202168A1
:1071C00048602046FFF794FF2068006810210840BF
:1071D000000900280BD020688068084000090028BA
:1071E00005D01020216848602046FFF73AFF20684C
:1071F000006820210840400900280BD020688068E2
:1072000008404009002805D0202021684860204619
:10721000FFF788FF206800684021084080090028A7
:107220000BD02068806808408009002805D04020E5
:10723000216848602046FFF774FF10BD70B5044612
:10724000002C01D1012070BD6068012800D100BF71
:1072500026496069884200D000BF2E20005D0028CA
:1072600005D100212D200155204600F059F80221BA
:107270002E2001552068C5686068012803D0890563
:10728000A06A884203D11E21284688430546174933
:107290006069884201D01648054016480540A1683B
:1072A00060680843216A0843616A0843A16A084389
:1072B00005436068012804D00121C905A06A8842FD
:1072C00003D1E168206908430543084960698842A1
:1072D00005D06169A0690843E16908430543206856
:1072E000C56001212E2001550020ACE7FFFF000002
:1072F0003F1FFFFFF8F119FF10B50446064920684B
:10730000884208D10548806B4000400803498863E3
:107310000D2000F065F810BD007C00400010024018
:1073200010B504460949206888420DD10848806B91
:107330004905084306498863002201210D2000F019
:1073400067F80D2000F058F810BD0000007C0040E8
:107350000010024001460868C069704710B5034636
:1073600002242E20C4541448006824072043124CE1
:1073700020601868C0680124E40420431C68E060B1
:1073800018688068012420431C68A06018680069A0
:10739000012420431C6820611868816118684261DB
:1073A00018680069042420431C68206101242E20F1
:1073B000C454002010BD00000004014070470000CC
:1073C0000648406B01210843044948630846806B26
:1073D0000904084301498863704700000010024017
:1073E00000BFC206D20E01219140024A116000BFC7
:1073F0007047000080E100E000BFC206D20E01210C
:107400009140024A116000BF7047000000E100E0B7
:1074100070B504460D4616462946204601F01CFE6E
:1074200070BD0000024949688143014A51607047BC
:107430000070004003480068FF2101310843014902
:107440000860704700700040024949680143014AE2
:1074500051607047007000400748006802210843EF
:10746000054908600548006904210843034908618B
:1074700000BF00BF30BF70470070004000ED00E06B
:1074800010B5024600200E4B1868800880000346A5
:10749000134318460A4B18600A4B1B690424234304
:1074A000084C2361012901D130BF02E040BF20BF59
:1074B00020BF044B1B690424A343024C236110BD6D
:1074C0000070004000ED00E0F8B50446202120687F
:1074D000084020287CD120680840202800D100BF27
:1074E00000278148806B012109070840002805D149
:1074F0007D48806B08437C49886301277B4800688E
:10750000FF2101310840002816D17848006808435F
:1075100076490860FFF766FD064606E0FFF762FD64
:10752000801B642801D90320F8BD70480068FF2142
:10753000013108400028F1D06B4805680321090596
:107540000D4060680840A8420DD0091160680840ED
:10755000884208D1644800680121490408408842F3
:1075600001D10120E0E760484030006903210904AF
:1075700008400546002D3DD060680840A84239D03B
:10758000202120680840202834D157484030006925
:10759000032109048843054653484030006901210E
:1075A000C904084350494031086108460069012177
:1075B000C90488434C49403108610846056180157B
:1075C00028408915884215D1FFF70CFD064608E0D2
:1075D00039E0FFF707FD801B4549884201D90320A8
:1075E000A2E7414840300069012149020840400AB1
:1075F0000028EED000BF00BF0321090460680840E6
:1076000088420AD1384800680901884303221205DC
:107610006168114008433449086000BF3248403077
:107620000069032212046168114008432E49403169
:10763000086100BF012F05D12B48806B8905884365
:107640002949886300BF2078C007C00F002809D0EF
:1076500025484030C06880088000A168084322495E
:107660004031C860022120680840022809D11E4824
:107670004030C0680C218843E16808431A49403112
:10768000C86004212068084004280AD11648403008
:10769000C0680321890288432169084312494031A7
:1076A000C86008212068084008280AD10E484030E8
:1076B000C068032109038843616908430A494031CE
:1076C000C86080212068084080280AD106484030E0
:1076D000C068032189048843A169084302494031F5
:1076E000C860002020E70000001002400070004049
:1076F00088130000F8B504460D46002C01D1012086
:10770000F8BD79480068C007C00FA8420ED276487D
:107710000068400840002843734908600846006834
:10772000C007C00FA84201D00120E9E7022120686C
:107730000840022807D16D48C068F0218843A1683D
:1077400008436A49C8602078C007C00F00284CD0A1
:107750006068022809D16548006801214904084091
:10776000400C002824D10120CAE76068032809D111
:107770005E480068012149060840400E002817D1E4
:107780000120BDE76068012808D15848006804213D
:107790000840800800280BD10120B1E75348006859
:1077A000012149020840400A002801D10120A7E731
:1077B0004E48C06880088000616808434B49C86033
:1077C000FFF710FC0646606802280FD107E0FFF7BC
:1077D00009FC801B4649884201D9032090E74348B1
:1077E000C0680C2108400828F1D134E06068032803
:1077F0000FD107E0FFF7F6FB801B3D49884201D916
:1078000003207DE73948C0680C2108400C28F1D1DD
:1078100021E0606801280FD107E0FFF7E3FB801B40
:107820003349884201D903206AE73048C0680C21F7
:1078300008400428F1D10EE007E0FFF7D3FB801BDE
:107840002B49884201D903205AE72848C0680C21F7
:1078500008400028F1D124480068C007C00FA842A2
:107860000ED9214800684008400028431E4908609E
:1078700008460068C007C00FA84201D001203FE7BA
:10788000042120680840042808D11848C06807214E
:1078900009028843E16808431449C8600821206848
:1078A0000840082809D11148C0680721C902884347
:1078B0002169C90008430D49C86000F049F80B4927
:1078C000C968F022114009090A4A515CC8400A49B6
:1078D00008600020FFF7AAFB0746002F01D03846BA
:1078E0000EE700200CE700000020024000100240DC
:1078F00088130000DEBC0008780100200148006801
:10790000704700007801002000B5FFF7F7FF054938
:10791000C968072212021140090A034A515CC84093
:1079200000BD000000100240EEBC000800B5FFF7EB
:10793000E5FF0549C9680722D2021140C90A034A76
:10794000515CC84000BD000000100240EEBC0008C1
:10795000FEB52E48C7680C203840002845D00428C2
:1079600004D008280CD00C283ED10BE02748006832
:1079700010210840002801D0254C00E0254C41E0B2
:10798000254C3FE00F2080043840800C23490E5CDA
:10799000032080053840800D401C01901B48C068C2
:1079A000012109040840002807D01B4971430846FB
:1079B0000199FDF79DFB054614E01448006810216D
:1079C0000840002807D01249714308460199FDF785
:1079D0008FFB054606E00F49714308460199FDF704
:1079E00087FB05462C460DE000BF0848406807218C
:1079F00049030840400B00900098401C0121814041
:107A0000CC0300BF00BF2046FEBD000000100240B6
:107A100000093D000024F40000127A00F6BC0008C2
:107A2000FEB50446002C01D10120FEBDF848C66811
:107A30000C210E40C768012109040F402078C007BF
:107A4000C00F002872D0082E04D00C2E0FD108468B
:107A500087420CD1EE480068012149040840400CDF
:107A6000002863D06068002860D10120DDE700BFF6
:107A7000012109046068884205D1E548006808438F
:107A8000E349086027E005210904606888420ED1B7
:107A9000DF480068012189040843DD490860084681
:107AA0000068012109040843D949086013E0D84857
:107AB0000068012109048843D54908600846006828
:107AC000012109040840009000BFD14800688900E6
:107AD0008843CF49086000BF6068002813D0FFF7D3
:107AE00081FA054606E0FFF77DFA401B642801D9BC
:107AF00003209AE7C6480068012149040840400C69
:107B00000028F0D012E0FFF76DFA054606E0FFF717
:107B100069FA401B642801D9032086E7BC48006845
:107B2000012149040840400C0028F0D102212068BE
:107B3000084002287AD1E0680290042E03D00C2E6F
:107B400034D1002F32D1B2480068042108408008A7
:107B5000002804D00298002801D1012065E7AC4834
:107B600040681F2109028843216909020843A84986
:107B70004860084600680921884302990843A449DF
:107B80000860FFF7E5FEA249C968F0221140090923
:107B9000A04A515CC840A04908600020FFF746FA9F
:107BA00001900198002841D001983EE702980028F2
:107BB00024D09748006809218843029908439449D2
:107BC0000860FFF70FFA054606E0FFF70BFA401BC7
:107BD000022801D9032028E78D48006804210840C5
:107BE00080080028F1D08A4840681F210902884394
:107BF0002169090208438649486017E08448006803
:107C00004008400082490860FFF7ECF9054606E0AD
:107C1000FFF7E8F9401B022801D9032005E77C485B
:107C200000680421084080080028F1D11021206854
:107C30000840102867D1002E36D1754800684901E8
:107C40000840400A002804D0A069002801D1012082
:107C5000EBE66F484068072149038843216A0843DF
:107C60006B494860084640680002000A217F090607
:107C7000084367494860206A400B401C012181404D
:107C8000C8036349C968F02211400909614A515C7F
:107C9000C840614908600020FFF7C8F901900198C9
:107CA00000284BD00198C0E6A06900282CD0584885
:107CB0000068FF210131084355490860FFF792F938
:107CC000054606E0FFF78EF9401B022801D9032084
:107CD000ABE64F480068012149020840400A0028ED
:107CE000F0D04B484068072149038843216A084384
:107CF00047494860084640680002000A217F09069B
:107D000008434349486019E041480068FF210131B8
:107D100088433F490860FFF765F9054606E0FFF72D
:107D200061F9401B022801D903207EE6384800682B
:107D3000012149020840400A0028F0D108212068AA
:107D40000840082839D1606900281BD030484030ED
:107D50000069012108432E4940310861FFF742F9CB
:107D6000054606E0FFF73EF9401B022801D9032033
:107D70005BE627484030006902210840400800289F
:107D8000F0D01AE022484030006940084000204905
:107D900040310861FFF726F9054606E0FFF722F9B2
:107DA000401B022801D903203FE6194840300069F2
:107DB0000221084040080028F0D104212068084032
:107DC000042879D1002000901148806B8906084072
:107DD000002806D10E48806B08430D4988630120B6
:107DE00000900E480068FF210131084000281ED194
:107DF0000A480068084309490860FFF7F3F8054698
:107E00000EE0FFF7EFF8401B642809D903200CE6C9
:107E100000100240DEBC0008780100200070004025
:107E200085480068FF21013108400028E9D000BFE3
:107E3000FF210131A068884205D1804800690843CC
:107E40007E49086130E0A06800280DD17B480069B8
:107E5000FF21013188437949086108460069091505
:107E60008843764908611FE005210902A06888421D
:107E70000DD1724800690121890208436F490861E8
:107E800008460069891508436C4908610CE06B4895
:107E90000069FF210131884368490861084600698B
:107EA000091588436549086100BFA068002815D0FE
:107EB000FFF798F8054608E031E0FFF793F8401B1C
:107EC0005F49884201D90320AFE55C480069012180
:107ED00049020840400A0028EFD013E0FFF782F87B
:107EE000054607E0FFF77EF8401B5549884201D957
:107EF00003209AE551480069012149020840400ADF
:107F00000028EFD10098012808D14C484038806BF8
:107F100001210907884349494039886300BF606AE5
:107F200000284CD00C2E69D0606A022848D1434802
:107F300040380068012109068843404940390860FB
:107F4000FFF750F8054606E0FFF74CF8401B022803
:107F500001D9032069E53948403800680121490604
:107F60000840400E0028EFD1E16AA06A0843216B67
:107F7000084332494039C968FD221204914308433D
:107F80002E494039C86008460068012109060843A7
:107F90002A4940390860FFF725F8054606E0FFF753
:107FA00021F8401B022801D903203EE52348403830
:107FB0000068012149060840400E0028EFD038E053
:107FC0001E48403800680121090688431B49403992
:107FD0000860FFF707F8054606E0FFF703F8401BC7
:107FE000022801D9032020E5144840380068012107
:107FF00049060840400E0028EFD11AE0606A0128C7
:1080000000D112E50D484038C7680120000438400F
:10801000A16A88420BD10F2080043840E16A88426F
:1080200005D1032080053840216B884201D0012012
:10803000FBE40020F9E40000007000404010024022
:108040008813000010B50446002C01D1012010BD9A
:10805000606A002800D100BF0021A1625120005DAC
:10806000002804D150200155204600F035F80221A7
:10807000512001552068006840218843216808602C
:10808000A16860680843E1680843216908436169A1
:10809000084301225202A16911400843E1690843E3
:1080A000216A0843A16A084321680860A069000C9E
:1080B00004210840616A0843216848602068C0695B
:1080C000910088432168C86100206065012151202A
:1080D00001550020BBE7000010B586B0044614210E
:1080E00001A8FDF778F814492068884222D1134886
:1080F000406B891408431149486300BF0846C06AB1
:10810000012108430D49C8620846C06AC007C00F74
:10811000009000BF00BFE0200190022002900020EC
:108120000390032004900020059001A9052000077A
:10813000FEF752FE06B010BD0030014000100240B4
:1081400070B504462546681E0949884201D90120B8
:108150000CE0681E074948610321081F00F07CFFFE
:1081600000200449886107200861002070BD0000DC
:10817000FFFFFF0000E000E070477047FEB50446D7
:108180002068C56920680668206887682807000F8E
:108190000190019800280ED12020284000280AD004
:1081A00020203040002806D0206E002802D0204633
:1081B000216E8847FEBD019800287DD0F807C00FCA
:1081C000002804D1FF20213030400028F5D0E807F6
:1081D000C00F00280BD0FF2001303040002806D00F
:1081E000012021680862E06F01210843E067022056
:1081F000284000280AD0F807C00F002806D0022027
:1082000021680862E06F04210843E06704202840E9
:1082100000280AD0F807C00F002806D004202168E3
:108220000862E06F02210843E06708202840002828
:108230000ED020203040002803D1F807C00F0028BE
:1082400006D0082021680862E06F08210843E06733
:10825000E06F002846D020202840002809D02020A8
:108260003040002805D0206E002802D02046216E24
:108270008847E06F009020688068402108404028CF
:1082800004D0082100980840002826D0204602F09B
:108290000EF82068806840210840402819D12068E5
:1082A0008068884321688860E06E00280DD02548EA
:1082B000E16E8863E06E00E015E0FEF763FB0028E6
:1082C00010D0E06E816B88470CE02046FFF755FF29
:1082D00008E02046FFF751FF04E02046FFF74DFF7E
:1082E0000020E06766E701200005284000280CD048
:1082F000012080053840002807D0012000052168B2
:1083000008622046FFF738FF54E780202840002805
:108310000AD080203040002806D0606E002802D0AD
:108320002046616E884745E740202840002807D056
:1083300040203040002803D0204601F0CAFF39E732
:1083400000BF37E7EDA1000810B50446002C01D1AD
:10835000012010BDA069002800D000E000BF606FC0
:10836000002805D1002170200155204600F02CF88E
:108370002420606720680068400840002168086089
:10838000204602F00DF8012800D1E2E7606A0028DB
:1083900002D0204601F09CFD206840680921C902F6
:1083A000884321684860206880682A2188432168C2
:1083B0008860206800680121084321680860204621
:1083C00001F0FEFDC5E7000010B586B0044614219B
:1083D00001A8FCF700FF36492068884266D135487D
:1083E000406B0121890308433249486300BF0846B6
:1083F000C06A012108432F49C8620846C06AC00705
:10840000C00F009000BF00BF032040020190022077
:10841000029000200390032004900420059001A9FD
:1084200005200007FEF7D8FC2348244908600320F4
:108430004860002121488160C160802101610021E4
:10844000416181612021C16100210162FEF74CFB85
:10845000002801D0FDF754FC00BF1848E066846294
:1084600000BF1548143816490860032048601021E1
:10847000134881600021C1608021016100214161B8
:108480008161C1610162FEF72FFB002801D0FDF779
:1084900037FC00BF0A48A066846200BF00220121A9
:1084A0001B20FEF7B5FF1B20FEF7A6FF06B010BD90
:1084B000003801400010024030000240341B002010
:1084C0007C1B002070B504460D461646A06F202880
:1084D00063D1002D01D0002E01D1012070BD0121FA
:1084E0000903A068884208D12069002805D1E8075F
:1084F000C00F002801D00120F0E700BF7020005D10
:10850000012801D10220E9E701217020015500BFB7
:108510006565582006530020E0672220A067E06EC2
:10852000002820D01E48E16EC8621E48E16E086334
:108530001D48E16E48630020E16E88632368194698
:1085400024313346626DE06EFEF722FB00280AD02C
:108550001020E06700BF00217020015500BF2020DF
:1085600060670120BAE700BF00217020015500BFFD
:1085700020680068FF2101310843216808602068F5
:108580008068012108432168886020688068402154
:108590000843216888600020A0E702209EE70000D1
:1085A00057A20008A1A2000805A200087047704762
:1085B000FFB583B004460D461746606F202875D17D
:1085C000002D01D0002F02D1012007B0F0BD012104
:1085D0000903A068884208D12069002805D1E8076E
:1085E000C00F002801D00120EFE700BF7020005D20
:1085F000012801D10220E8E701217020015500BFC8
:108600000020E06721206067FEF7ECFC019050201D
:1086100007535220075301210903A068884205D15E
:108620002069002802D10026029502E02E46002093
:10863000029021E006980090002280212046019BB4
:1086400002F09CF8002801D00320BEE7002E09D1DB
:1086500002980088C005C00D216888620298801CBD
:10866000029003E0307821688862761C5220005B1B
:10867000401E81B2522001535220005B0028D9D104
:1086800006980090002240212046019B02F076F8D7
:10869000002801D0032098E72020606700BF002158
:1086A0007020015500BF00208FE7FFE702208CE714
:1086B000704700BFFEE710B5002204210520000727
:1086C000FEF789FC0022082105200007FEF783FC45
:1086D0000A2002F0DBFB0122042105200007FEF73F
:1086E0007AFC0A2002F0D2FB0022042105200007B8
:1086F000FEF771FC10BD10B5002204210520000713
:10870000FEF769FC0122082105200007FEF763FC43
:108710000A2002F0BBFB0122042105200007FEF71E
:108720005AFC0A2002F0B2FB0022042105200007B7
:10873000FEF751FC10BD70B50546002400261EE072
:108740000022042105200007FEF745FC0A2002F064
:108750009DFB0122042105200007FEF73CFC60067A
:10876000040E082105200007FEF72CFC002801D08C
:10877000601CC4B2052002F089FB701CC6B2082E32
:10878000DEDB002D02D1FFF7B6FF01E0FFF793FF1C
:10879000204670BD70B50446002204210520000764
:1087A000FEF719FC00252AE080202040C011002897
:1087B00006D00122082105200007FEF70CFC05E089
:1087C0000022082105200007FEF705FC6006040EC4
:1087D0000A2002F05BFB0122042105200007FEF7BE
:1087E000FAFB0A2002F052FB0022042105200007B8
:1087F000FEF7F1FB0A2002F049FB681CC5B2082D08
:10880000D2DB70BD10B50122082105200007FEF75C
:10881000E2FB0122042105200007FEF7DCFB002219
:10882000082105200007FEF7D6FB0A2002F02EFBE8
:108830000022042105200007FEF7CDFB10BD10B576
:108840000022042105200007FEF7C5FB00220821B5
:1088500005200007FEF7BFFB0A2002F017FB0122EC
:10886000042105200007FEF7B6FB012208210520A0
:108870000007FEF7B0FB0A2002F008FB10BD10B5A0
:1088800000240122082105200007FEF7A4FB062092
:1088900002F0FCFA0122042105200007FEF79BFBF1
:1088A000062002F0F3FA07E0601CC4B2FA2C03DDE4
:1088B000FFF7C5FF012010BD082105200007FEF7C6
:1088C00081FB0028F0D10022042105200007FEF7DB
:1088D00082FB0020EFE7000038B501F0A9FB01F0B2
:1088E000FBFB5A480068C06908210840002802D0F4
:1088F00057485849C860FDF755FB0446564800786C
:10890000002806D001280AD0022819D0032824D133
:108910001DE0012291025148FEF75DFB1DE0FF20A2
:10892000F530844206DA0022012189024B48FEF725
:1089300052FB04E0012291024848FEF74CFB0CE098
:108940000022012189024548FEF745FB05E001228E
:1089500091024248FEF73FFB00BF00BF0121C90260
:108960003E48FEF72FFB00281BD03D4800786328C7
:108970000BDD0022012149033848FEF72CFB0122C0
:1089800011033648FEF727FB17E001225103334855
:10899000FEF721FB0022012109033048FEF71BFBF3
:1089A0000BE00022012149032C48FEF714FB0022B2
:1089B000012109032948FEF70EFB2A48808C012873
:1089C00020D100252848009072B680212748FDF765
:1089D000B3F90546002D05D0022269462348FDF76C
:1089E0009DFA054662B622A001F0FEFF00211D4857
:1089F000818403F0E3F8642002F03EFA144815493C
:108A0000C86000BF1748408C01280ED100211548CE
:108A10004184002013494039088003F0CFF86420D6
:108A200002F02AFA0A480B49C8600E48008C012857
:108A30000AD100210B48018403F0C0F8642002F041
:108A40001BFA03480349C86038BD0000B41A00206F
:108A50000400FA0500ED00E032010020000400509F
:108A600048010020EC0D0020AAAA0000384A0008A6
:108A7000BDF8C8EBC9FDBCB6C4A3CABD0D0A000051
:108A800008B53721202000F073F80321212000F0E1
:108A90006FF84021222000F06BF80821232000F01D
:108AA00067F8AA21302000F063F80A48008FC1B2AD
:108AB000322000F05DF80221332000F059F85F21E8
:108AC000202000F055F8684600F006F80A2002F071
:108AD000DDF908BDAC0D002010B5044621460F207D
:108AE00000F023F8002800D110BD0120FCE770B58C
:108AF00004460025FFF786FE3220FFF74BFEFFF706
:108B0000BEFEE0B2FFF746FEFFF7B9FEFFF77AFEC2
:108B10003320FFF73FFEFFF7B2FE0020FFF70BFE0A
:108B20000546FFF78CFE284670BD70B505460C461D
:108B30002846FFF7DCFF2070012070BD70B50446A9
:108B40000D46FFF75FFE3220FFF724FEFFF797FE8A
:108B5000E0B2FFF71FFEFFF792FE2846FFF71AFE6E
:108B6000FFF78DFEFFF76BFE0A2002F08FF970BD54
:108B700070B504460D4629462046FFF7DFFF012069
:108B800070BD000010B50248FEF7CDFA10BD000020
:108B90002C1A0020F0B585B004460020039072B670
:108BA0004F4920684018002806D14E48C06803216C
:108BB00089040840039000E000BF00BF206880687F
:108BC00002902068C0680190206845692068866925
:108BD00043492068401800280DD142484038806A37
:108BE000490508433F49403988620846806A400089
:108BF0004008886200E000BF00BF002D01D1002EB8
:108C00005FD0374920684018002807D13548C06830
:108C10000321890488433349C86000E000BF00BFD6
:108C2000002D1DD0206800690121084321680861DA
:108C300020684561FEF7D6F9074600BFFEF7D2F976
:108C4000C01B00902068006808210840082804D054
:108C50007D21C90000988842F0D908202168486029
:108C6000002E1DD020680069012108432168086199
:108C700020688661FEF7B6F9074600BFFEF7B2F935
:108C8000C01B00902068006810210840102804D004
:108C90007D21C90000988842F0D9102021684860E1
:108CA0000F4920684018002809D10E48C0680321E8
:108CB00089048843039908430A49C86000E000BF5B
:108CC00000BF2068006940084000216808610298E0
:108CD0002168886001982168C86062B605B0F0BD5F
:108CE0000084FFBF401002401CB50020009001909E
:108CF0001E481F49086000211D48C16301208007EC
:108D00001B49486000211A488160072181630121C5
:108D100001610021C160001D01774177001F816260
:108D2000FF21C23141620021243001720421243824
:108D300041610021016381614163C161FDF722FC52
:108D4000002801D0FCF7DCFF0A4800908013019056
:108D500069460748FDF78AFB002801D0FCF7D0FFE1
:108D600000210348FDF714FB1CBD00000024014056
:108D7000D01900200200000408B500BF0A48006BAB
:108D800001210843084908630846006BC007C00F6B
:108D9000009000BF00BF002201210A20FEF738FB2F
:108DA0000A20FEF729FB08BD0010024000B587B07D
:108DB000142102A8FCF70FFA00BF6548C06A04211D
:108DC00008436349C8620846C06A0421084001900C
:108DD00000BF00BF00BF5E48C06A802108435C49F5
:108DE000C8620846C06A80210840019000BF00BFE9
:108DF00000BF5748C06A012108435549C862084668
:108E0000C06AC007C00F019000BF00BF00BF084686
:108E1000C06A022108434E49C8620846C06A02215E
:108E20000840019000BF00BF01224A490520000709
:108E3000FEF7D1F8012291024748FEF7CCF8002254
:108E400046494548FEF7C7F800228121090205205E
:108E50000007FEF7C0F8012002904148039000206F
:108E6000049002A905200007FDF7B6FF022002903A
:108E7000032003900020049002A905200007FDF7BD
:108E8000ABFF0C20029011200390002004900320DF
:108E9000059002A905200007FDF79EFF2120000193
:108EA000029001200390002004900220059002A966
:108EB00005200007FDF790FF01200290112003908C
:108EC00000200490059002A92348FDF785FF0220A9
:108ED0000290244803900120049002A91E48FDF747
:108EE0007BFF214802900120039000200490059010
:108EF00002A91948FDF770FF0120C002029000206E
:108F000003900220049002A91348FDF765FF912009
:108F1000000202900120039000200490059002A915
:108F200005200007FDF758FF8020029000200390E5
:108F30000120049002A90848FDF74EFF00220121FC
:108F40000520FEF765FA0520FEF756FA07B000BDCA
:108F5000001002401C100000000400500930000006
:108F600000001110000021100834000010B50A485C
:108F70000A490860002048600021084881600849CB
:108F800041610021016241628162FEF757F90028C8
:108F900001D0FCF7B5FE10BD007C00402C1A00206B
:108FA000FFFF000010B5124812490860FF2005308D
:108FB000486000210F488160C16001614161012169
:108FC000490281610021C161016241628162072120
:108FD000C162FFF737F8002801D0FCF791FE054881
:108FE000006800684021084302490968086010BD14
:108FF000003001405C1A002010B513481349086086
:10900000E12040024860002110488160C160016198
:109010000C21416100218161C161016200200B4985
:1090200048620846FFF790F9002801D0FCF768FE77
:10903000C82207490548FFF745FA002801D0FCF788
:109040005FFE01F0DDFB10BD00380140B41A0020C6
:10905000E40C00207047000010B5002819DA1A4A05
:1090600003071B0F083B9B089B00D2588307DC0EAD
:10907000FF23A3409A438B071B0E8407E40EA340F3
:109080001A43114B0407240F083CA408A4001A51EA
:1090900018E00E4A03231B02D21883089B00D25803
:1090A0008307DC0EFF23A3409A438B071B0E840724
:1090B000E40EA3401A43054B032424021B19840821
:1090C000A4001A5110BD00001CED00E000E100E01A
:1090D00000BF00BF00BFBFF34F8F00BF00BF00BF86
:1090E00006480749C86000BF00BF00BFBFF34F8FED
:1090F00000BF00BF00BF00BF00BFFDE70400FA05CE
:1091000000ED00E0F0B593B000200E90962002F044
:1091100035FA4B20C00002F04DFA0020FE490870DD
:10912000FE4800780C2802DB0B20FC490870012265
:10913000510205200007FDF74EFFF8480078F84976
:109140000870F6480078F74908700020F649087062
:10915000FDF77EF8F5494870F54801780068401C35
:10916000F34A1060C8B2F149C870EE4800788872BE
:10917000EC4800784200EF49EC480B30FCF712F85D
:109180000620EA4948720846EB490A784270497855
:109190008170E4490978490008460D300022E3490E
:1091A00002F00AFBDF490978490008460D3000212A
:1091B00002F016FB022002F03BFA0020DF490870A3
:1091C0000120DF4908700020DE490870DE48FEF704
:1091D000C1F8DE4908800020D3490870D1480078E2
:1091E000FCF73AFA0646FCF7B7FAD94AD94B05918B
:1091F0000490FCF751F90791069001F0D9FD002287
:1092000001239B0709910890FCF794F80B910A90B1
:10921000FCF784FAC0B20D900D984001CB49098843
:109220004018CD490880084600880121C9038842BA
:1092300004DBC9480088401AC7490880C748C849A4
:109240000860C8480078401CC6490870BE48FEF750
:1092500081F8C549088070E2BB48FEF77BF8C24937
:10926000088033E0B548007800281BD002F042F9AE
:10927000109012991098884214D911991098884228
:1092800010D201F0B5FF0020AD490870384602F059
:109290006DF9012002F0CCF9B44908700020A7490B
:1092A00008701DE0A848FEF755F8AF490880084649
:1092B0000088A9490988884208DBAB480088A6498C
:1092C0000988AB4A8918884200DA09E000210F209A
:1092D00002F0ACF8A7490860A74908400028C1D0AF
:1092E00000BFA4480068401C002801D1FFF7F0FE31
:1092F000A048006801218903084000287ED081220F
:10930000D20100210F2002F010FA0021102002F0FB
:109310008DF84006400E0F90002298480F9902F0F9
:10932000D5F8002002F046F9002002F0F2F8934848
:10933000407A07288FD1022291499048401DFBF7BF
:1093400055FF002887D102F0A8FA8E4A03C202F026
:109350008DFA8D4A03C274480078401C7249087027
:109360008648427808A90A74807848746C48007866
:10937000002810D10120854908706846008E6D498B
:109380000880012067490870684908A8007C487077
:1093900008A8407C8870674800886946098E884222
:1093A0007DD17B497548C08908807A487349098A0C
:1093B00001806548FDF7CEFF6B490880754800883D
:1093C000FF30C330734908800846008872498842DC
:1093D00012DD70480088401A6E4908806C48008889
:1093E000401C6B490880084600886B490B31884255
:1093F00002DB002066490880002600E091E105209C
:109400006649885566495D4842890A808089488056
:1094100008460068B100634A50505848C07C624911
:10942000087000204F4908700120444908704C49D9
:10943000524842890A80808948803A480078FF2152
:1094400091314843FF309B30FF30F5300004C117A5
:109450004D4B0CCB801859410906070A0F4353485E
:10946000381A129019208002381811907908490092
:1094700000200A0E000210430B02002211469A1827
:1094800048414B490A6048603E480CC827480A30AA
:1094900002F0D2F93C480CC82448163000E0EBE05A
:1094A00002F0CAF942480CC82048123002F0C4F950
:1094B00008201E4948721B490978890008461C305B
:1094C00000221A4902F078F91649097889000846FD
:1094D0001C30002102F084F901201A49087004228E
:1094E0002649491C3348FBF75DFE002032490880BD
:1094F000274800887D21C90048432649098840182B
:109500002E4908602E4800782E4908702E49C888D8
:10951000FCF7A2F8049059E0E90000202A0100209D
:109520002901002028010020090100202016002028
:109530006C0000201A180020020100201C010020ED
:109540001E0100201D0100202C1A002022010020F5
:10955000333333333333E33F24010020A08601004B
:10956000040100201901002020010020E800002053
:10957000983A00007000002000D0272470160020C8
:109580003C01002078000020800000201B0100200A
:1095900044010020F4000020E7030000DC18002054
:1095A000F80000204C180020320100200052030077
:1095B000880000202C0100204A0100200C0100201E
:1095C000620100202B010020AC0D0020E348008840
:1095D000FCF742F803900499FBF76EFE0590FCF748
:1095E000BBF80791069002F09BFA0022DC4B099130
:1095F0000890FBF79FFE0B910A90FCF78FF8D94972
:109600000880D9480078401E0988884202D101208C
:10961000D6490870D1480088D5490880D54900202E
:10962000085EFCF721F809910890D3480088FCF700
:109630002FF8D24AD24B01910090FBF72DFF0591F4
:109640000490D0480068FCF70FF803910290059B46
:10965000049AFBF713FF07910690099B089AFBF702
:1096600069FE0B910A90FCF735F8C7490860C748B6
:10967000008800F013FB53E06846008EFCF77CFC8A
:109680000646C34909788E4213DB0120C1490870A0
:10969000C1480078401CC04908706846008E7100BF
:1096A000BE4A5052BE4908A8007C487008A8407CB9
:1096B00088700520BB498855BB49BC4842890A804F
:1096C0008089488008460068B100B94A5050B748C0
:1096D000C07CB8490978884207DDB448C07C0328BB
:1096E00003D0B248C07CB3490870B0001630AC4912
:1096F00040180B90B0480CC80B9802F09DF8A64992
:109700000978890008461C300022A54902F054F867
:10971000A1490978890008461C30002102F060F850
:109720000BE0A64A00210F2001F0FFFFA4480078BB
:10973000002802D0002001F0ECFE8F480088A149EB
:109740000988884200DA87E58B4800889D490988A6
:109750009D4A89188842F6DC984A00210F2001F0C2
:10976000E4FF9A4800788C49087000258D480078FD
:10977000002814D196480068FCF70AFD9549088036
:1097800008880988491E934B198093490988FBF77B
:10979000C5FC92480088414388B27C49088000207B
:1097A0008F490870002423E07E48005D00281DDDFD
:1097B0008B480078401C8A4908707A48005DA900EF
:1097C000884A505060007549085A6900864A5052CC
:1097D000A00077490A582846691CCDB28000834909
:1097E0000A507048005D401E6E490855601CC4B2A6
:1097F00067480078674909784018A042D4DC73486C
:109800000078032803DA76480078754908707448B0
:1098100000785F49087000243FE0002536E0A8008A
:1098200072490958681C8000704A105881422BDD2B
:10983000AA006E4B99586A006B4B985AA200694B6C
:109840009A580C926A1C9200684B9A58AB00674E6B
:10985000F2506A1C5200644B9A5A6B00624EF252EC
:109860006A1C92005F4B9A58AB005E4EF2506A1C25
:1098700092005E4B99506A1C52005B4B98526B1CD5
:109880009B000C9AF25000BF681CC5B2404800789B
:10989000401EA842C3DC601CC4B23D480078401E94
:1098A000A042BADC002052490870002438E0600071
:1098B0004D49085A6100394A5052A0004B49085896
:1098C000A1003B4A5050A00011460858494988421F
:1098D00024D0A000434908580A281FD144480078E2
:1098E00006214843001D4449401861002B4A89184D
:1098F0000A78027049784170A2002D4BD1183C4A79
:10990000127806235A43921D3B4BD0180422FBF7D2
:1099100049FC37480078401C35490870601CC4B2C7
:109920001B4800788442C2DB002405E03148A100D6
:109930001F4A5050601CC4B20C2CF7DB1F4A803207
:1099400000210F2001F0F1FE002201214902052033
:109950000007FDF740FB13B0F0BD000044010020FC
:109960000000F03F620100202B0100201D010020BB
:10997000260100203001002020010020F853E3A53B
:109980009B843E400C010020140100204A0100206D
:10999000290100201B010020280100201A180020A6
:1099A00020160020DC180020F8000020701600208F
:1099B0004C180020320100208000002000D0272415
:1099C0001E01002024010020983A00000901002017
:1099D0002C010020FC000020500100204E0100203E
:1099E0002A010020AC180020321800207C1800202A
:1099F0001A010020FFFF0100CE1700207047000071
:109A0000F0B585B047484849086002F015F8FF20D6
:109A10000B30464948800846C08E45490870434887
:109A2000C08F444908704148808F434908703F48BF
:109A3000807A424908703D488088414908603B4926
:109A40000889FBF725FE044600223E4BFBF78CFD00
:109A50000191009001F0ACF906460022394BFBF76A
:109A600069FC03910290FBF759FE374908802F49A2
:109A7000C88835490988FBF751FB344908802B49D0
:109A8000888832490988FBF749FB2F480088414301
:109A900088B22F49088009887D22D20051430846A8
:109AA000FBF7E2FD06462B4A2B4BFBF75DFD044618
:109AB000FBF734FE2949088025480088284908809A
:109AC0001A48C1887D20C000FBF728FB2549088083
:109AD0001648C1887D20C000FBF720FB2249088082
:109AE000012022490880FCF75DFA214908801B48C3
:109AF000028820492048FDF731FC002801D0FCF7FE
:109B0000FFF80F4801681DA000F06EFF0748C188EC
:109B10001EA000F069FF0548018921A000F064FF44
:109B200005B0F0BD0DA8000848000020AC0D0020D5
:109B3000010000205E0100205F010020470100209D
:109B40003C010020000010404E0100205001002088
:109B50004A010020F853E3A59B843E4056010020B3
:109B60005A010020580100206001002062010020FD
:109B70005C010020FF7F00002C1A0020B1EAC7A979
:109B800049443A202564202E0D0A0000CDA8D1B604
:109B9000BCE4B8F43A202564206D732E0D0A000051
:109BA000B5A5B4CECDA8D1B6BBF9D5BECAFDC1BF4F
:109BB0003A202564B8F62E0D0A00000000B585B0E5
:109BC00014216846FBF707FB00220121C903104856
:109BD000FDF701FA0120C003009001200190002050
:109BE0000290039069460A48FDF7F6F80120C00389
:109BF00000900320019000200290039069460448E1
:109C0000FDF7EAF8022001F037F905B000BD0000C9
:109C1000000400507047000038B504460D4600208F
:109C2000009055201B490870AA20487003208870B6
:109C3000601DC87003200871084645718471680072
:109C4000154A811822461348C01DFBF7ABFA0020C5
:109C500008E0811C0F4A525C6946098851188AB293
:109C60000092401C611D8842F3DB0A48801CFBF710
:109C700097FF0090E01D074941186846007808707A
:109C800068464078487021460931024800F03AFBA6
:109C900038BD00006C190020AC0D0020F0B585B077
:109CA000054600251A4800881A490988884206DBBB
:109CB0001748008817490988401A1549088016482E
:109CC000C08813490988484347197D21C9004F437B
:109CD000124800683E1A3046FBF7C6FC104A114B8A
:109CE00001910090FBF740FC03910290FBF7F2FC1E
:109CF00004460D498C4201DD0846241A002C01DA85
:109D00000948241809480068446105B0F0BD000006
:109D10006201002060010020AC0D00201401002031
:109D2000F853E3A59B843E40FF7F00002C1A0020DF
:109D300001460020054A126890B2054A10400246CA
:109D40000A431046014A106070470000003001408D
:109D5000C7FF000010B5FDF74BF910BD00B599B075
:109D600034210CA8FBF737FA142107A8FBF733FAC4
:109D70001C216846FBF72FFA244800680321C9021A
:109D800088430121C902401820490860FDF752FBB1
:109D90001F4800690321C90288431D490861062044
:109DA0000C9088150E9001200F901020109002202A
:109DB00015900021169141041791410518910CA8A6
:109DC000FDF72EFE002801D0FBF79AFF0F20079029
:109DD00003200890002009900A900B90012107A809
:109DE000FDF788FC002801D0FBF78AFF8120009056
:109DF000002002900320800406906846FDF764FB73
:109E0000002801D0FBF77CFF19B000BD00700040B6
:109E10004010024015480068FF21013108431349F2
:109E200008600846C068124908401049C8600846E2
:109E30000068104908400D490860084680684008DD
:109E4000400088600846006801218904884307496A
:109E500008600846C068FD21090488430349C860BA
:109E600000200861044805498860704700100240DE
:109E70000C40FF88F6FFF6FE0050000800ED00E001
:109E800010B501F0EDFA044602E001F0E9FA0446EB
:109E90000C488442F9D100200B4908800B48007817
:109EA000002804D0012803D0022807D103E005E0F0
:109EB000FCF79AF802E0FFF725F900BF00BF01F0B8
:109EC0007BF910BD3001CADEE600002060000020F2
:109ED000818CC907C90F002908D00168496801228F
:109EE00052049143826A1143026851600222416A1E
:109EF0001140022907D101684968D2039143C26A1F
:109F00001143026851600422416A1140042907D1BB
:109F10000168496812049143026B11430268516061
:109F20000822416A1140082907D1016849681203D3
:109F30009143426B1143026851601022416A114003
:109F4000102907D10168896812029143826B11437D
:109F5000026891602022416A1140202907D10168DE
:109F6000896812029143C26B1143026891604022DA
:109F7000416A1140402915D1016849689203914313
:109F8000026C11430268516001221205016C91427A
:109F900008D101684968032252059143426C11437C
:109FA000026851608022416A1140802907D101680E
:109FB000496812039143826C1143026851607047F3
:109FC00038B504460020E067FDF70CF80546206828
:109FD00000680821084008280BD114482B460022AD
:109FE00089040090204600F0C9FB002801D003201E
:109FF00038BD206800680421084004280BD10B48B4
:10A000002B46002209050090204600F0B7FB0028EF
:10A0100001D00320ECE720206067A06700BF00218B
:10A020007020015500BF0020E2E70000FFFFFF01A4
:10A0300070B50025C82420480078002800D070BDE5
:10A040001E480078002800D0F9E701201B4908705D
:10A050001B48406B002801D10870F0E71848406B9E
:10A06000C8210D1A1CE01749174A1268885C174965
:10A0700009688847164800883C21484315490880EC
:10A0800011480068401C1049086008460068C8284C
:10A0900001DB002008600A48406BC8210D1A641ECD
:10A0A00009480068A84201D0002CDCDC00200349EC
:10A0B000087000BFC3E700004200002044000020F9
:10A0C00000000240E40C002038000020480000207E
:10A0D000580100206801002010B53A480078002897
:10A0E00003D139480078002800D010BD012036493E
:10A0F00008703648C06980210840002802D13249E2
:10A100000870F2E7324900200856324900228A5688
:10A11000904215D12D48C0694021084000280BD03D
:10A120002D480078002807D000202B4908702B48C4
:10A130000088401C29490880002023490870D4E782
:10A1400025480078002805D10120234908700A20FD
:10A1500000F09CFE1F4900200856CC2148432049AE
:10A160004018001D1F490968405C184988621D4855
:10A170000068401C1B490860164900200856CC2185
:10A1800048431749085817490968884214DC0020D9
:10A19000144908600F480078401C40B20D4908700F
:10A1A000084600780E2801D1002008700E4800787B
:10A1B000401C40B20C49087000200349087000BFE1
:10A1C00093E70000420000204300002000380140D7
:10A1D00035000020340000204500002052000020FF
:10A1E000BC010020580000203600002070B5054654
:10A1F000AC6A00215A200153522001532046FDF73A
:10A20000BCFF70BDF8B50546AC6A666FA76F2068E5
:10A21000806880210840802807D1212E05D10021A7
:10A2200052200153204600F064F8206880684021E5
:10A230000840402807D1222F05D100215A20015380
:10A24000204600F034F8E06F10210843E067204614
:10A25000FDF793FFF8BD70B50546AC6A2868006845
:10A2600020210840002817D100215A2001532068DE
:10A270000068FF21013188432168086020688068F8
:10A280004008400021688860206880684021884339
:10A29000216888602020A0672046FEF787F970BDFE
:10A2A00070B50446A56A2846FEF781F970BD0168BD
:10A2B0000968FF22213291430268116001688968B0
:10A2C00049084900026891602021816700210166E8
:10A2D000704710B504462068006840218843216813
:10A2E000086020206067002060662046FEF7E0F9E5
:10A2F00010BD01680968C0229143026811602021E5
:10A300004167704770B505460C4620480078002824
:10A3100003D11F480078002800D070BD01201B49E0
:10A320000870C82C04DC1B4800214156002903DCBE
:10A33000002016490870F0E7174900200856CC2184
:10A34000484316490C50144A00215156CC2251431F
:10A35000124A8918081D22462946FAF723FF0E489B
:10A360000078401C40B20C490870084600780E285E
:10A3700001D10020087007480078401E40B205490E
:10A38000087000200149087000BFC6E742000020A5
:10A39000430000203600002035000020BC010020D2
:10A3A000F0B587B0044610200490002500200390EB
:10A3B0000026E7492068884200D100E000BF2169FB
:10A3C000A068084361690843E169084307462068BB
:10A3D0000068E04908403843216808602068406808
:10A3E000032109038843E168084321684860A7699D
:10A3F000D7492068884201D0206A074320688068D6
:10A400000B210902884338432168886000BFD24984
:10A41000206888421CD1D148C0688007800F00287E
:10A4200006D001280AD0022805D003280CD108E064
:10A43000012004900BE00220049008E00420049026
:10A4400005E00820049002E01020049000BF46E0E0
:10A45000C349206888421CD1C048C0680C2108400C
:10A46000002806D004280AD0082805D00C280CD1D2
:10A4700008E0002004900BE00220049008E0042093
:10A48000049005E00820049002E01020049000BF32
:10A4900025E0AF49206888421FD1B048C068032139
:10A4A00089020840002808D001218902401A0AD0F8
:10A4B000401A05D0401A0CD108E0002004900BE0AF
:10A4C0000220049008E00420049005E00820049095
:10A4D00002E01020049000BF01E01020049000BFB3
:10A4E0009B492068884256D1049804281AD004DC7D
:10A4F000002807D002281CD108E0082816D0102810
:10A5000017D117E0FDF700FA064616E093484038E9
:10A510000068102108400009002801D0914E00E099
:10A52000914E0AE0FDF714FA064606E00126F6030E
:10A5300003E000BF0120039000BF00BF002E0AD03F
:10A54000606841004018B04203D860680003B04220
:10A5500002D201200390F4E0606802903046FF21AF
:10A56000013100F068FA62685208002380185941EE
:10A5700001910090029AFAF7E5FD054603200002DA
:10A58000854205D37948854202D82068C560D8E065
:10A5900001200390D5E00121C903E06988426FD111
:10A5A000049804283CD006DC002809D0012813D0E8
:10A5B00002284AD11CE008283ED0102845D145E0A9
:10A5C000FDF7A2F9400061684908401802906168EF
:10A5D000FAF78EFD85B23CE0FDF7A8F9400061680E
:10A5E0004908401802906168FAF782FD85B230E0B0
:10A5F0005A4840380068102108400009002807D058
:10A6000061684A085A4BD018FAF772FD85B206E025
:10A6100061684A08574BD018FAF76AFD85B218E00E
:10A62000FDF796F94000616849084018029061689A
:10A63000FAF75EFD85B20CE061684A0801231B044D
:10A64000D018FAF755FD85B203E000BF0120039052
:10A6500000BF00BF102D0FD3474885420CD8464895
:10A660000F38284005902807400F059908430590AA
:10A6700005982168C86064E00120039061E0FFE76D
:10A68000049804283AD006DC002809D0012812D00A
:10A69000022847D11AE008283BD0102842D142E0D6
:10A6A000FDF732F961684908401802906168FAF7CD
:10A6B0001FFD85B23AE0FDF739F961684908401895
:10A6C00002906168FAF714FD85B22FE02348403804
:10A6D0000068102108400009002807D061684A0876
:10A6E000204BD018FAF704FD85B206E061684A08ED
:10A6F0001D4BD018FAF7FCFC85B217E0FDF728F9DE
:10A7000061684908401802906168FAF7F1FC85B267
:10A710000CE061684A080123DB03D018FAF7E8FC73
:10A7200085B203E000BF0120039000BF00BF102DE1
:10A7300005D31148854202D82068C56001E0012098
:10A740000390002020666066039807B0F0BD00000B
:10A7500000480040F369FFEF00380140401002401C
:10A760000044004000093D000024F400FFFF0F00FA
:10A7700000127A000048E801FFFF0000FFB581B039
:10A7800004460D4617460A9E22E0701C00281FD082
:10A79000FCF728FC0499401AB04201D8002E17D1CA
:10A7A00020680068FF21A131884321680860206883
:10A7B0008068400840002168886020206067A067AA
:10A7C00000BF00217020015500BF032005B0F0BD7F
:10A7D0002068C0692840A84201D1012000E0002083
:10A7E000B842D2D00020F1E710B510200349096823
:10A7F00008620248FDF7C2FC10BD0000B41A002038
:10A800000D200149087070473600002070B50446DD
:10A8100000256A480078082865D100BF002004E0C0
:10A820006749095C49198DB2401C66490978491F7E
:10A830008142F5DC64480078281885B261480078C8
:10A84000281885B261480078281885B260480078D9
:10A85000281885B25F480078281885B26019C007AB
:10A86000C00F002835D058480078012827D002288A
:10A870002DD15949554A1278881855490A785049B6
:10A88000FAF790FC01F09AF9642000F0F5FA00BFA5
:10A8900000BF00BF00BF00BFBFF34F8F00BF00BFAE
:10A8A00000BF4E484E49C86000BF00BF00BFBFF3A5
:10A8B0004F8F00BF00BF00BF00BF00BFFDE7434890
:10A8C0000078411042480078FFF7A6F900E000BF89
:10A8D00000BF0020394908703C49087039490870A8
:10A8E0004049087068E035480078072812D134489C
:10A8F0003C49097844543B480078401C3949087069
:10A9000030480078401F0978884255D108202B49EB
:10A91000087051E029480078062805D12C480470B9
:10A9200007202649087047E024480078052805D10B
:10A93000264804700620214908703DE01F48007831
:10A94000042805D12048047005201C49087033E014
:10A950001A480078032808D11A48047000201B49BF
:10A96000087004201549087026E014480078002873
:10A9700005D1552C03D10120104908701CE00F4867
:10A980000078012805D1AA2C03D102200B490870B8
:10A9900012E00A480078022807D1032C05D10320D1
:10A9A000064908700B48047006E00020034908704F
:10A9B000064908700349087070BD0000340100208A
:10A9C000081900203601002039010020370100203D
:10A9D0003501002038010020AC0D00200400FA05EC
:10A9E00000ED00E03A0100200FB410B503A9044BBC
:10A9F000044A029800F034F910BC08BC04B01847AF
:10AA000055B800087C0100202021020C01D0102143
:10AA10001046020A01D010460839020901D010463A
:10AA2000091F820801D01046891E420801D0881EE5
:10AA30007047081A7047F8B582B28BB2040C0D0C3F
:10AA400010465843002126465E43370C36048019D1
:10AA5000794116466E43370C3604801979412646F3
:10AA60006E438919F8BD30B47446641E2578641CA1
:10AA7000AB4204D3635D5B00E31830BC18471D464E
:10AA8000F8E702E008C8121F08C1002AFAD170478F
:10AA90007047002001E001C1121F002AFBD170475E
:10AAA00008B5002100916B46012202212C2000F004
:10AAB00051FE022100916B4601222C2000F04AFE3B
:10AAC00008BD000038B504466D2000906B46012299
:10AAD00008492E2000F03EFE002C05D0064A07490A
:10AAE0002E2000F011FE04E0054A04492E2000F05B
:10AAF0000BFE38BD0608000007060000061800001F
:10AB00000716000038B504466B46022200213620A5
:10AB100000F0ACFC2300FFF7A6FF0E11081A5454F6
:10AB20005454233154543D444B5400216846017021
:10AB30004078FE2108406946487043E0694608783D
:10AB4000FC21084001210843694608703AE0694643
:10AB50000878FC210840022108436946087031E06A
:10AB600068460078B32108404821014368460170D7
:10AB70004078802108436946487023E068460178A0
:10AB8000B32001406846017040784106490E68468E
:10AB9000417017E0694648780221084369464870C9
:10ABA00010E069464878FD2108406946487009E090
:10ABB00069460878CF21084020210843694608707B
:10ABC00000E000BF00BF6B4601220021362000F0EC
:10ABD000C1FD00AB013301221146362000F0BAFD61
:10ABE00038BD08B5032168464170012101706B46EC
:10ABF00002220021362000F0ADFD0122D203062101
:10AC00002D2000F081FD012000F036F90120FFF732
:10AC100079FF08BD38B504462004010E684641702E
:10AC200004706B46022204212D2000F093FD0321C5
:10AC3000684601706B46012206212D2000F08AFD36
:10AC40000021684601706B46012206212D2000F08C
:10AC500081FD0A212D2000F0E9FB0546284638BD7C
:10AC6000FFB58DB00446002506E025280AD0109ACD
:10AC70000F999047641C6D1C20780028F5D1284658
:10AC800011B0F0BD00270121484A009700E00743BA
:10AC9000641C23780846203B98401042F7D1207866
:10ACA0002E2817D1042007436078641C2A280CD171
:10ACB0000E98641C02C800910E900BE000990A22C5
:10ACC000514330394018641C0090207801463039D7
:10ACD0000929F3D920780028D1D0642808D0692820
:10ACE00006D075281ED0109A0F9990476D1C5BE016
:10ACF0000A200E99019001C90E91002802DA404203
:10AD00002D2102E0390504D52B216A46117201215B
:10AD100003E0F90704D02021F7E70BAE0B910DE01B
:10AD20000021FAE70A200E99019001C90E91F7E778
:10AD30000199FAF7DDF93031761E31700028F7D12C
:10AD400003A8801B20300190780701D5009801E00E
:10AD5000012000900199884201DD401A00E00020A6
:10AD60000027009006E002A8109AC05D0F99904756
:10AD70006D1C7F1C0B988742F5DB04E0109A302095
:10AD80000F9990476D1C0099481E00900029F5DC32
:10AD900005E03078109A761C0F9990476D1C019948
:10ADA000481E01900029F4DC641C65E709280100B5
:10ADB000F8B54A002B4B520DD6182B4A0C460546C7
:10ADC000142E2BDA002E12DA284BFAF7B3FA0022EF
:10ADD0001346FAF7D5FC40D2002C03DA0124E4072D
:10ADE00000253AE02046284337D0214C14E0214F7B
:10ADF0000B46F7403B402B4331D01C4BFAF79AFAF5
:10AE000000221346FAF7BCFC27D2002C03DD0120F8
:10AE10000005F0400419BC4300251EE0332E1EDC63
:10AE200033460027143BFF43DF40384217D00F4B17
:10AE3000FAF72AFB00221346FAF7A2FC0DD2002CE7
:10AE40000ADD142E0CD03420811B012088404019CB
:10AE5000A84200D2641C0546BD4321462846F8BDE1
:10AE6000641CF9E701FCFFFF9C7500883CE4377E19
:10AE70000000F03FFFFF0F0070B504467D20C000CA
:10AE800060430546284600F001F870BD002100BF70
:10AE900040E000BF00BF00BF00BF00BF00BF00BF59
:10AEA00000BF00BF00BF00BF00BF00BF00BF00BFAA
:10AEB00000BF00BF00BF00BF00BF00BF00BF00BF9A
:10AEC00000BF00BF00BF00BF00BF00BF00BF00BF8A
:10AED00000BF00BF00BF00BF00BF00BF00BF00BF7A
:10AEE00000BF00BF00BF00BF00BF00BF00BF00BF6A
:10AEF00000BF00BF00BF00BF00BF00BF00BF00BF5A
:10AF000000BF00BF00BF00BF00BF00BF00BF00BF49
:10AF100000BF491C8142BCD370470000F0B585B02A
:10AF200004460020049003902578607940008A4907
:10AF3000085A02906078401E8849C6B20863042D02
:10AF400001D0072D01D1012000E0002001902078E0
:10AF500082490873E07900280AD1084680690121F6
:10AF6000890508437D4988610298C010029006E077
:10AF70007A48806901218905884378498861207A67
:10AF80007649487308468069217A0904032212042D
:10AF900011400843714988610846002182690420F4
:10AFA00000F0C3FB6E492E20029A00F0ADFB304644
:10AFB000FFF788FD6B48405D810040186A494318DF
:10AFC000052207212B2000F0C5FB684901980B18CA
:10AFD00001220B21282000F0BDFB6248405D80006B
:10AFE00063490A580C21282000F09FFBE07980007B
:10AFF00060494018A1794900425A0221272000F0F7
:10B0000083FB70005C490A5A0421272000F07CFB76
:10B01000E079002805D164220621272000F074FB86
:10B020001EE0A07804280DD11020009010220621E7
:10B03000272000F069FB6B4601222621272000F023
:10B0400089FB0DE02820009020220621272000F017
:10B050005BFB6B4601222621272000F07BFB00BF13
:10B06000300146494018E1788900425808212720DC
:10B0700000F05BFBA17A627A08021043002803D13A
:10B080003F496172090AA172A17A637A08021843E2
:10B0900002462021272000F037FB3A480C210268A5
:10B0A000232000F042FB71003648001D425A042163
:10B0B000232000F029FBA07900280BD0E079324949
:10B0C000431801220021212000F044FB03200490BA
:10B0D000012003902807000F2901F02211400843A6
:10B0E00061788904032292041140084304990905F8
:10B0F000920011400843039949040122520411406F
:10B100000843217989051F2292051140084361797E
:10B11000C906C90EC906084307463A4600211F2042
:10B1200000F003FBA0786178084300040B49086134
:10B1300008460069E17949030122D203114308431B
:10B1400006490861084600210269082000F0EDFA6E
:10B15000002005B0F0BD0000ACBC0008800100205C
:10B160000428000054BC0008020000202000002039
:10B170005CBC00087CBC000888BC00088CBC0008D3
:10B180004110000074BC00082200002038B50446BD
:10B190000D460848808B0443224600212C2000F0F5
:10B1A000B3FA00956B46012206212C2000F0D2FA5A
:10B1B00038BD00008001002010B5FFF771FC10BD04
:10B1C00070B505460421362000F030F90446002D04
:10B1D00003D00120C002044304E00121C90220463B
:10B1E0008843044622460421362000F09EFA70BDB2
:10B1F00038B54020009000210E2000F017F90446D9
:10B20000002211460E2000F090FA6B460122002128
:10B210000D2000F09FFA084A00210F2000F085FA67
:10B2200000F056FA224600210E2000F07EFA00219E
:10B230000248017338BD0000F8FF2724A001002058
:10B24000F0B585B00646042002900027002001904A
:10B2500066494875086300216448203041710173D4
:10B260000020624988834863886300F0F9F85F49E9
:10B27000086003E000F0F4F85C4908605B4800688F
:10B280005B498842F6D10020FFF73CFC5948007822
:10B29000432802DD432057490870564800780028AB
:10B2A00002DA00205349087052480078242804DD4F
:10B2B000504800780446243C0DE006214D480078B3
:10B2C000F9F72CFF0621081A45014A480078F9F7DA
:10B2D00025FF2C460C432006210408432102084385
:10B2E0002043039000211E20039A00F01EFA02ABB7
:10B2F00001220021242000F02DFA1E20FFF78AFCF5
:10B3000087B23812394988730420FFF783FC019013
:10B310000198C0B200280FD0022000906B46012295
:10B3200012212D2000F016FA3048808B01210903EC
:10B3300008432E49888300BF00F092F82B4908602B
:10B340000620FFF767FC294948600720FFF762FCE9
:10B3500026498860F806C00E08750846007D00285A
:10B3600001D1102008752149087D00F04BFAF00743
:10B37000C00F002809D0FFF734FC1C48808B012146
:10B38000C9020843194988830CE00521362000F0E2
:10B3900035F80546184805402A460521362000F0B4
:10B3A000B3F900BF0120FFF7ADFB0021042000F03E
:10B3B0003DF80E4988610021262000F037F8054647
:10B3C000052080030543800005432A4600212620EE
:10B3D00000F0ABF900222621362000F095F900F0AC
:10B3E0003FF802490860002005B0F0BD8001002050
:10B3F0003001CADE01000020FFFD0000F8B5044660
:10B400000D46094FA9B2A0B26B46022200F02EF8F9
:10B410000646002E06D1684640780102684600784C
:10B42000081887B23846F8BDFFFF0000FEB5054694
:10B430000E460027FF43B1B2A8B201AB042200F0D0
:10B4400015F800900098002808D1032404E0380281
:10B4500001A9095D4718641E002CF8DA3846FEBDC4
:10B4600010B500210846FFF7E1FF10BDFFB581B020
:10B4700006460C4617460025002C04D129466D1CB3
:10B48000684646541AE040203043C2B229466D1C3B
:10B49000684642547F2C04DC28466D1C69460C54D7
:10B4A0000CE0E0B28021084329466D1C6A465054E6
:10B4B0006004020E28466D1C69460A54A8B23A463A
:10B4C0006946049B00F0F8FA05B0F0BD70B504467B
:10B4D0000D46164623462A4631461120FFF7C6FF81
:10B4E00070BD10B504462346052200211520FFF744
:10B4F000BDFF10BD10B501210620FFF797FF10BD5D
:10B5000010B504462346052200211720FFF7AEFFA1
:10B5100010BD38B504460020009000F0D9F8FF2592
:10B520000135002C01D0680005432A4600210D207A
:10B5300000F0EAF8002C17D06B46012203210F20FF
:10B54000FFF794FF684600780821084000280BD0D8
:10B55000FFF74EFEFF2501352A4600210D2000F0A1
:10B56000D3F80020C04338BD0020FCE710B50446E6
:10B57000224601210A2000F0D8F810BD70B505461A
:10B5800000211A20FFF752FF0446240D240528034A
:10B59000000B0443224600211A2000F0C6F870BDBB
:10B5A00010B50446224602492E2000F0ADF810BD29
:10B5B0000418000038B504466B460122032104201C
:10B5C000FFF754FF002C16DD224600210C2000F06E
:10B5D0009BF8694608781021084300900F4880695D
:10B5E000090608430D4988616B46012203210420A6
:10B5F00000F0B0F810E06946087810218843009008
:10B600000648806909068843044988616B4601221F
:10B610000321042000F09EF838BD000080010020C6
:10B6200010B5044622460021182000F06DF810BD28
:10B63000F8B5044600250020009000260220204096
:10B6400000280AD0802000906B46012200210D20A6
:10B6500000F080F801211D480173E007C00F0028A9
:10B6600026D0694608780621084300906B460122DF
:10B6700000210D2000F06EF803210F20FFF7BEFE21
:10B6800006468120C0003040002801D100251AE084
:10B69000402000906B46012200210D2000F05AF856
:10B6A0000020FFF78DFD0021084801734D1E0AE0C0
:10B6B000694608780221084300906B460122002168
:10B6C0000D2000F047F82846F8BD0000A00100203A
:10B6D0001CB501AB012203210F20FFF7C7FE69460D
:10B6E00008798021084069460979402211404900C3
:10B6F000884208D0012000906B46012203210D20D2
:10B7000000F028F800BF1CBDF8B505460E461446EB
:10B710006846047021124170B1B2A8B26B46022291
:10B7200000F018F807463846F8BDFEB506460F4645
:10B730001446002503E069464C55240A6D1C042D6F
:10B74000F9DBB9B2B0B26B46042200F003F8019005
:10B750000198FEBDFFB581B006460C461746002590
:10B76000002C07D180203043C2B229466D1C6846A8
:10B77000425419E0C0203043C2B228466D1C6946CD
:10B780000A547F2C03DC28466D1C0C540CE0E0B2FC
:10B790008021084329466D1C6A4650546004020EFD
:10B7A00028466D1C69460A54A8B23A466946049B6D
:10B7B00000F01EFA05B0F0BD70B504460E46154601
:10B7C000281901218902884202DD0020C04370BD92
:10B7D000A21E334629460920FFF7BCFF0020F6E7EA
:10B7E00070B504460D46064800692043A905084384
:10B7F0000646324600210820FFF797FF002070BD63
:10B800008001002038B504466B4601220E212B2012
:10B81000FFF72CFE68460078410949010091E106D6
:10B82000C90E68460078014300916B4601220E2143
:10B830002B20FFF78FFF38BD70B50146002006E0D2
:10B840000A541E06140A34431B0A2246401C0428CC
:10B85000F6DB70BD13B50C4601231A466946024853
:10B86000FCF7A6FE00981CBDB41A00207CB5002190
:10B870000C460D466846FFF734FE042608E0220E0B
:10B8800028021043240205466846805D0443761E64
:10B89000002EF4DA204629467CBD7CB500210C46FA
:10B8A0000D466846FFF72CFE042608E0220E28020B
:10B8B0001043240205466846805D0443761E002E30
:10B8C000F4DA204629467CBDFBF79AFBFEF746FAE0
:10B8D000FDF76CFAFDF74AFBFDF78EFBFDF762FB07
:10B8E000FDF702FAFDF748FAFEF78AF8FDF7C8F807
:10B8F000FAF7C6F9FAF788F90721FF204130FFF778
:10B9000045FCFFF759FC012028490880012201036A
:10B9100005200007FBF75FFB46E02548007800287C
:10B9200040D0FEF71BFA002021490870FAF790FC7E
:10B9300020490870084600780F280FDD0122D10346
:10B9400005200007FBF747FBFEF79AFA00220121CA
:10B95000C90305200007FBF73EFB0BE0012208218D
:10B960001548FBF738FBFEF78BFA00220821124836
:10B97000FBF731FBFCF7B0FF0C480088002804DD22
:10B980000A480088401E094908800C4800780028B1
:10B990000AD106480088002806D101210846FBF795
:10B9A0006FFD01E0FCF798FFB7E700006801002099
:10B9B00049010020480100200004005045000020FB
:10B9C00000B585B01748FBF794FB14216846F9F7DA
:10B9D00002FC154800900320019000200290694667
:10B9E00005200007FBF7F8F969461048FBF7F4F962
:10B9F00069460F48FBF7F0F901210846FBF740FDC7
:10BA0000FF200130FBF70EFD0A48006804210843BF
:10BA1000084908608815FBF717FDFBF71DFD05B009
:10BA200000BD00002C1A0020FFFF000000040050A1
:10BA3000000800500070004010B50122D2021B49DE
:10BA40001B48FAF794F9194800881A4988422CD003
:10BA5000084616490880042088807D20C000C880E0
:10BA600001200881002048811E20C04388810120D8
:10BA7000C88100200884088248828882C88208839E
:10BA800088834320C88601200887782048870120C2
:10BA90008887C8870021054840300184418481841B
:10BAA00000200249C88300F089F810BDAC0D0020C9
:10BAB00000F00008AA55000070B504460D460021AC
:10BAC000102005263607B06200BF0DE0685C134EFB
:10BAD000F06000BF11488068C007C00F0028F9D08F
:10BAE0000E48C0681870491CA142EFDB00210DE030
:10BAF00000200A4EF06000BF08488068C007C00FF1
:10BB00000028F9D00548C0685854491C9142EFD329
:10BB1000102005263607B061002070BD00300140BE
:10BB2000F0B513B406460199F9F742FF04460D46F5
:10BB300002460B4630460199F9F7A0FC06460198EB
:10BB40001B4B0F4600280CDA00223046F9F76EFF37
:10BB50000CD90022174B30463946F9F711FE1DD299
:10BB600014E000223046F9F761FF08D20022124BA0
:10BB700020462946F9F782FC04460D460EE00022D5
:10BB80000C4B30463946F9F7FBFD07D800220A4B2B
:10BB900020462946F9F7CEFB04460D46019A690076
:10BBA0004908D20FD2072046114303B0F0BD000070
:10BBB0000000E0BF0000E03F0000F03F10B50024AF
:10BBC00072B60121C9020848FAF7B6F80446002CFB
:10BBD00006D00122D20205490348FAF79FF904462C
:10BBE00062B6204610BD000000F00008AC0D002039
:10BBF00070B504460D460021102005263607B062B8
:10BC000000BF0CE0685C124EF06000BF1048806816
:10BC1000C007C00F0028F9D00D48C068491CA142D8
:10BC2000F0DB00210CE0585C094EF06000BF0848D2
:10BC30008068C007C00F0028F9D00548C068491CBB
:10BC40009142F0D3102005263607B061002070BD68
:10BC5000003001400000010203040005405C0000C8
:10BC6000A05C0400C06C0800805C0400E03F1E0083
:10BC7000E07D1E0007A9022570889B880A00160037
:10BC8000010006000100020087008D002D001A311E
:10BC900052001A339A001A351D011A376B003B31D6
:10BCA000BE003B335E013B3596023B37000099599D
:10BCB0009959EB518F421E45142E0080EB51F52807
:10BCC0003333E13A703DE13AC235852BC235333327
:10BCD000C235C235AE47E13A5138A3305138000081
:10BCE000000000000000010203040607080900002C
:10BCF000000001020304030406080C1018203000A1
:10BD000020BD00080000002080010000785A0008D3
:10BD10005CBD000880010020601E000092AA00089F
:10BD200021130704380D091E080540082609104094
:10BD300008560A131D043B08BE0596D8BC401008DF
:10BD4000042FC8420115010202141309091202024C
:0CBD5000C5816B8C0AD901405220000014
:04000005080050C1DE
:00000001FF
